:020000020000FC
:0200000054C1E9
:10006800DF93CF934F933F932F931F930F93CC27F7
:1000780040E2DD27000F111F221F331FDD1FDA307A
:1000880010F0DA5003954A95A9F7DA30D05DDF937E
:10009800C395071517052705370551F700E3C33042
:1000A8001CF40F93C395FBCF0F91AFD5CA95E1F719
:1000B8000F911F912F913F914F91CF91DF9108950B
:1000C8000F93012F01D00F91029501D002950F9344
:1000D8000F700A3008F0095F005D97D50F910895F9
:1000E80000E293C51F930F930E9499000D008F01A2
:1000F800E7DF10E1F5DF183009F4F2DFF1DF0191F5
:10010800E3DF1A95C1F77097EBDFEADF10E10191A1
:10011800003210F00F3708F00EE277D51A95B9F7CC
:100128007097DEDF0F911F910895FF93EF93DF9390
:10013800CF930F93DEB7CDB7EF81FE81EE0FFF1F90
:100148000591003031F061D50D30D1F70AE05DD569
:10015800F7CF3196F695E795EF83FE830F91CF9110
:10016800DF91EF91FF910895115030F009910590BA
:10017800001919F40020C1F7001B0895042F77D047
:10018800D4DF202041203D00092D9EDFCEDF204214
:1001980043203D001881098193DFC7DF20444520B3
:1001A8003D001A810B818CDFC0DF20484C203D00C8
:1001B8001C810D8185DFB9DF2053503D0000870188
:1001C8007FDFB3DF2050433D00008C0179DFADDFD6
:1001D8002020202020202000DC010E94690774DFF5
:1001E800A4DF20000E9469076FDF9FDF20000E94C4
:1001F80049076ADF9ADF20000C8539D096DF202076
:1002080061273D000D8560DF90DF206263273D0098
:100218001E810F8155DF89DF206465273D00188521
:1002280009854EDF82DF20686C273D001A850B8523
:1002380047DF7BDF2049583D00001E850F8540DFE2
:1002480074DF2049593D00001889098939DF6DDFBD
:1002580020493D000A8938DF68DF2020202020203F
:1002680020000895535A204820564E4300001F93FB
:10027800102F5BDF0D00EF93FF93ECE6F2E00591A2
:10028800002339F0003219F017FF00E2BED4111F25
:10029800F6CFFF91EF911F9108950000FEFCF8F44E
:1002A800FF000FEF0DBF08E00EBFE2EAF2E0C0E08A
:1002B800D0E0B591B993EA3AE1F7A89574BE08E1A0
:1002C8000093600000E10093600000E105BF6BB897
:1002D80065B868B86AB864B867B8209870926F0053
:1002E800709270007092B0007092B100E0E0F1E09E
:1002F80014E07192E139F107E1F700E21EE410938E
:100308008B0000938A0001E80093810000916F0040
:10031800046000936F000FD30EE40093B3000091C4
:10032800B00002600093B0000091B1000260009339
:10033800B100009170000260009370007894E9D4D5
:10034800E7D10AE06CD1F1DE0D0D43504D206F6E00
:1003580020616E204156522C2076332E3100E5DE86
:100368002072323031200000E0DE0D00DEDE546500
:100378007374696E672052414D3A2066696C6C2E21
:100388002E2E0000A0E0B0E00B2F0A27A4D5E0F73E
:10039800CCDE776169742E2E2E0018E00FEF3FD166
:1003A8001A95E1F7C2DE7265726561642E2E2E0021
:1003B800A0E0B0E02227F894BBB928B8ABB938B8A8
:1003C8007AB848B800C0000009B168B878946AB82B
:1003D8001B2F1A27011731F1222349F4A6DE0D003D
:1003E800A4DE4164647220787820797920009DDE4B
:1003F8000D00302F8D0164DE7FD00B2F0A27102FC0
:1004080063DE7AD0032F60DE77D0012F0327012324
:1004180078D072D0012F03271095012372D023952D
:10042800203110F4119638F6222351F07EDE205345
:10043800797374656D2068616C7465642100FFCF01
:10044800A0E0B0E006E747D5E8F76FDE0D006DDE07
:10045800496E6974696E67206D6D632E2E2E0000DB
:1004680064DE0D000E94C70B0F7729F55EDE4E6F24
:1004780020626F6F7461626C652043502F4D206459
:1004880069736B20666F756E642120506C656173AB
:1004980065206368616E6765204D4D432F53442D79
:1004A800436172642E0041DE0D0012E10FEFB7D0F8
:1004B8001A95E1F7CACF0E941F0C37DE0D0035DE12
:1004C80050617274696E697420646F6E652E0000E5
:1004D8000E94B10A7092F4017092F5017092F601CF
:1004E8007092F701A0E0B0E2A093F901B093FA018D
:1004F8000E94B80A0C94620F0F9300E286D30F9102
:1005080008951F932F93102F28E00DE2110F08F480
:0E05180008E57BD32A95C9F72F911F9108950E
:02001C0084C29C
:10052600409B1895419840980000409A4098419AFF
:04053600409A18953A
:0200300084C288
:10053A00EF93EFB7EF93FF93E0918A00F0918B006E
:10054A00E05EF14BF0938B00E0938A00CF93DF9348
:10055A00C0E0D1E0E0912301E15020F0E0932301D3
:10056A0009F408D3E881E15008F0E883E981E15011
:10057A0008F0E983EE85FF853196EE87FF87E83E2E
:10058A00E3E0FE07F4F17E867F86E889F9893196F1
:10059A00E88BF98B29F4EA89FB893196EA8BFB8B84
:1005AA00EB8DE395EB8FEC3360F17B8EEC8DE3956D
:1005BA00EC8FEC3330F17C8EED8DE395ED8FE831E5
:1005CA0000F17D8E0F93E9E1F6E00F8DE00FF71D44
:1005DA00F491023021F4E8A1E37009F4F395EE8D69
:1005EA00E395EE8FFE1760F4E1E0EE8F03950F8F2F
:1005FA000D3030F0EF8FE8A1F9A13196E8A3F9A305
:10060A000F91DF91CF91FF91EF91EFBFEF91189585
:10061A001F1C1F1E1F1E1F1F1E1F1E1F00930001CF
:10062A00009100010030E1F70895E4E1F1E02223AE
:10063A0021F0E20FF71D0081089527E0F894078161
:10064A0001932A95E1F778941291029132D00083AE
:10065A00118325E0029122D000832A95D9F70091CF
:10066A0014010895E4E1F1E0E20FF71D008322236B
:10067A0009F0089525E0008134D001932A95D9F72D
:10068A000081118139D00193119327E0F8940291E6
:10069A0007832A95E1F778947AD008951F931AE090
:1006AA00062C0394011BE8F7010F0294000D1F9119
:1006BA00089520E1080100271127000C111C001FD2
:1006CA00111F2A9569F01D5F13FF1350105D17FF64
:1006DA0010530D5F03FF0350005D07FF0053EDCF7A
:1006EA0008951F93102F12951F700F70012E1AE094
:1006FA00109D000D1F910895F4DF0F93012FF1DF74
:10070A0014E6019F0F91112D000D171D08957F9278
:10071A007F927F927F9200E10F93FEB7EDB700EAD6
:10072A000F9312E010D313E027D300234AF121815B
:10073A00328112E0118307D316E01ED3002302F19F
:10074A000481001F001F001F0227037011F0239568
:10075A00371DABE1B1E0F8940181C3DF0D9302814B
:10076A00C0DF0D930381BDDF0D9304810F73B9DFE1
:10077A000D9305810F71B5DF0D932D933D937894F9
:10078A000F910F910F910F910F910F910895EBE136
:10079A00F1E0F894108121813281A3810481C5811D
:1007AA00D68178947BDF0F930A2F78DFAC2FA2953E
:1007BA00AA0FAA0FA07C0A2B0F93032F6FDF0F93A8
:1007CA00022F6CDF0F93012F69DF0F937F9204E8EA
:1007DA000F937F92FEB7EDB700EA0F9319E0B3D2F9
:1007EA0004E0028313E0AFD2D383C28300E1018322
:1007FA0014E0A9D2E85FFF4FF894EDBF7894FEBFEA
:10080A0008950FEFE8E0F1E0215020F021F0E20F27
:10081A00F71D0081089516E0F894068101931A9550
:10082A00E1F77894009108010895215060F40130AD
:10083A00D9F0023031F00F3009F1003109F45AC011
:10084A0008951CD011C0E8E0F1E021F0E20FF71D95
:10085A00008308950083359616E0F8940681019383
:10086A001A95E1F778940895E2E0F1E016E0F89439
:10087A00048501931A95E1F778940895DF93CF934D
:10088A00E2E0F1E0F894C4851191C11BD48511917D
:10089A00D10B18F4C851DC4F0894DF93CF93048529
:1008AA00C1910C0B1485D1911D0B2485C1912C0B80
:1008BA0078943485D1913D0B37DC0D0035DC5469D1
:1008CA006D65722072756E6E696E672E20456C6159
:1008DA00707365643A200000C2DB26DC2E000F919B
:1008EA001F9120E030E0BBDB1FDC732E0000CF91AC
:1008FA00DF910895EEE0F1E0F89401910F930191F0
:10090A000F93019111912191789431910DDC0D0091
:10091A000BDC557074696D653A200000A0DB04DCBD
:10092A002C0020E030E01F910F9199DBFDDB732E44
:10093A0000000895219800EC10E8009380001093BD
:10094A008200219A00E206BB00916F0000620093C8
:04095A006F0008958D
:020028009AC478
:10095E000F930FB70F93FF93EF93E0918600F091F3
:10096E0087001F9310E400918100012700938100FE
:10097E0000E206BB009122010030C1F4E093250194
:10098E00F09326017092240101E00093220102E00F
:10099E0000932301189BA0C0E1E8E0938100F0E2F0
:1009AE00F6BB709222017092230196C00130C9F5F8
:1009BE000091250110912601E0932501F093260167
:1009CE00E01BF10BE755F040E0F000E8EE5AF04086
:1009DE0090F00695D8F7EE5AF04008F467C0709282
:1009EE0023017092220151607092290170922A01A6
:1009FE0070922B0171C00093240102E0009322013A
:100A0E006BC001E80093810000E206BB70922201E8
:100A1E000FE3F8D0E95AFF4F0F2F53DB0E2F51DBA8
:100A2E005BC0023009F50091250110912601E0937B
:100A3E002501F0932601E01BF10BE755F0400091E4
:100A4E0024010894079548F0EE5AF040D0F7009331
:100A5E00240103E0009322013FC011E01093220114
:100A6E0012E01093230126C00330C9F40091250132
:100A7E0010912601E0932501F0932601E01BF10B66
:100A8E00E755F04000912401069580F0EE5AF040B3
:100A9E00D8F70093240102E0009322011DC0E1E883
:100AAE00E0938100E0E27092220116C07092230161
:100ABE0070922201F0912901F03870F4F395F093C1
:100ACE002901EFE2F0912A01EF0FF395FF77F093F2
:100ADE002A01F1E0F71D00831F91EF91FF910F9115
:060AEE000FBF0F911895E7
:02002C0063C5AA
:100AF400EF93EFB7EF93FF93E0918800F0918900B3
:100B0400E255FF4FF0938900E0938800E0912701BC
:100B1400EA9512F5E0912C01EA95BAF0E0932C01E4
:100B24000F93EFEAF1E000912E01E00FF71D03951A
:100B34000F7100932E01008100950093280109E0B4
:100B4400009327010F91F0E811C0E0916F00ED7F51
:100B5400E0936F00F0EC0AC0E0932701F0E8E09125
:100B64002801E0FFF0ECE695E0932801F093800083
:100B7400FF91EF91EFBFEF911895709222010F93BF
:100B840000912401002341F4516070922901709274
:100B94002A0170922B0119C0E02FE095E0780695A8
:100BA4000E2BE8F7F0912901F03878F4F395F093DF
:100BB4002901EFE2F0912A01EF0FF395FF77F0930B
:100BC4002A01F1E008F4F39500830F910895FF934F
:100BD400EF931F93009129010023E1F3EFE2F1E089
:100BE40010912B01E10FF71D13951F77F8940091D5
:100BF4002901015010F47894EDCF0093290110934A
:100C04002B01789400811F91EF91FF910895FF9338
:100C1400EF93EFB7EF930F9300912C010032E0F7BD
:100C2400EFEAF1E000912D01E00FF71D03950F713C
:100C340000932D010F910083F894F0912C01F3950A
:100C4400F0932C01F13091F4F0916F00F1FD0EC09E
:100C5400F260F0936F00E0918400F09185007E963D
:100C6400F0938900E0938800E2E0E6BBEF91EFBFE8
:100C7400EF91FF9108950F9300912C010023E1F768
:040C84000F9108952F
:0200600013C6C5
:100C88000F930FB70F931F93FF93EF93EFECF1E0E0
:100C980010810091B900083069F0003159F008312D
:100CA80051F0083241F00034C9F0003589F00835B8
:100CB800F1F023C011270281101740F4E10FF71D4E
:100CC800139503810093BB0005E818C0718215C015
:100CD800E10FF71D13950091BB0003830091D1012B
:100CE8000A95101710F405EC09C005E807C07182D1
:100CF800E10FF71D0091BB00038304E90093BC00DA
:100D08001093CF01EF91FF911F910F910FBF0F919A
:100D180018950CE50093B8006092BB0004E00093BE
:100D2800BC007092D00108950EE10093000100917B
:100D3800BC00017139F0009100010023C1F70EEFEA
:100D48000093D00100230895EFDFB2F0FF93EF93F3
:100D5800BF93AF93A0EDB1E06D921D9301910E7F0B
:100D68000D931A9511F00191FBCF05EA0093BC0091
:100D7800AF91BF91EF91FF910895D6DFDAF0FF931D
:100D8800EF93BF93AF93A0EDB1E06D921D930081F7
:100D980001600C9305EA0093BC00C6DF0091D00106
:100DA80007FD04C00D9101931A95E1F7AF91BF912A
:100DB800EF91FF910091D00108950091D00108951D
:100DC800E4EEF1E0E20FF71D00810895E4EEF1E0B2
:100DD800E20FF71D00830895A7DFEAF0EFECF1E0DA
:100DE80061822091E40122833396A091E501B091BC
:100DF800E6010E946907016001932A9505EA0093BC
:100E0800BC0092DF0091D00107FD05C001910E944E
:100E18006F072A95D9F7089587DFBAF0EFECF1E06C
:100E280061822091E40122833396A091E501B0917B
:100E3800E6010E9469070E7F01932A9519F00E9426
:100E48006907FACF05EA0093BC000895013009F458
:100E5800C3CF023009F4E0CF08956F92FEB7EDB723
:100E680000E2020F000F0F9312E087DF0F910F913E
:100E780008950F93FEB7EDB700E2020F000F0F932E
:100E880012E062DF0F910F910895F894BBB928B86A
:100E9800ABB938B87AB848B800C0000009B168B82A
:100EA8006AB878940895F894BBB928B8ABB938B83B
:100EB8000BB958B868B878940895E7DF11960F937E
:100EC800E4DF1196102F0F910895DFDF1196089532
:100ED800EADF1196012FE7DF119608950093E701E5
:100EE8001093E80108953F932F932091E7013091E3
:100EF800E801020F131F30F00093E7011093E80197
:100F0800890102C0002711272F913F910895DC2FF6
:100F1800CB2FBA2FA0E0BB0FCC1FDD1F08956EBCEE
:100F28000DB407FEFDCF0EB508950EBD0DB407FE36
:100F3800FDCF08951F9312E0F2DF60920101EFDF09
:100F4800061511F401E006C0009101010030B9F75F
:100F58001A9599F71F91002308952A9AE0DF002730
:100F680008952A98E7DFC9F30F6F089517FF13C094
:100F7800DF93CF93BF93AF931F93C0E0D0E0DE0120
:100F880017E3F4DF1F91AF91BF91CF91DF9102304A
:100F980010F000230895E1DFE4DF11F40FEF1EC025
:100FA800012F0F770064C1DFDEBDC0DFCEBDBEDF1D
:100FB800BEBDBCDFAEBDBADF05E9103021F007E8E1
:100FC800183009F001E0B1DF1C3009F4A8DF0AE0AD
:100FD800102EA5DF07FF02C01A94D9F70023089541
:100FE800C5DF0E1739F414E0EAE1F0E098DF019369
:100FF8001A95E1F7089500910001002329F43A9524
:1010080019F004E60093000108950091E9010160D8
:101018000093E90103E50CBD7DBC1AE080DF1A9559
:10102800E9F720E010E0C0E0D0E0DE019FDF01300A
:1010380009F03AC03AE004E60093000118E0C0E085
:10104800D0E0B1E0AAEAE1E0CBDFB9F4C130A9F41D
:10105800DA3A99F419EAD0E4C0E0B0E0A0E086DF1B
:1010680019F0C9DFE1F708C01AE3D0E0E0E0B8DF23
:1010780019F42460A6FD286017C019EAC0E0D0E082
:10108800DE0174DF023018F4226019EA02C0216020
:1010980011E06CDF19F0AFDFE1F706C010E1A0E066
:1010A800B2E064DF09F020E02093EA0156DF009106
:1010B800E901222319F00E7F0093E9017CBC089511
:1010C800E1E5F2E00090E90103E001FC089500E5A4
:1010D8000CBD01E00DBD0091EA0103FF18DF11E12D
:1010E80045DF11E0E9F4C0E0D2E008EC009300012C
:1010F80016DF061521F4009000010714C9F70E3F0A
:1011080079F40DDF6EBC219739F001930DB407FE19
:10111800FDCF0EB56EBCF7CF019308DF00DF10E0FE
:101128001CDF7CBC012F08950090E90103E001FC5D
:10113800089500E50CBD01E00DBD0091EA0103FF33
:10114800E6DE11E113DF11E079F5C0E0D2E008EC4A
:1011580000930001E4DE061521F41091000110301F
:10116800C9F70E3F11E001F5DADE6EBC2197C9F030
:10117800E715F70539F031970DB407FEFDCF0EB529
:101188006EBCF4CFE02F0DB407FEFDCF0EB56EBCDC
:10119800F02F219731F00DB407FEFDCF0EB56EBCD0
:1011A800F8CFC4DEBCDE10E0D8DE7CBC012F089589
:1011B800E1E5F2E00090E90103E001FC089500E5B3
:1011C8000CBD01E00DBD0091EA0103FFA0DE18E1AE
:1011D800CDDEB1F4AFDEA1F00EEF0EBDC0E0D2E07F
:1011E80001910DB407FEFDCF0EBD2197C9F79EDE14
:1011F8000FEF9BDE9ADE93DE0F71053010E009F0E9
:1012080001E0ABDE7CBC012F0895F9E0FE9FE9E028
:10121800F2E0E00DF11D0895E2EFF1E0E20FF71DB5
:101228000895FADF0083213031F00895223079F0F3
:10123800F3DF00810895A091F201B02FEBEEF1E009
:1012480026E043DE01932A95E1F75CD008951091DA
:10125800F1010091F4010830A8F4112339F452D0B7
:1012680092D20F931F911F770091F401011740F458
:1012780047D0012B21F42091F401022FF5D00895D5
:1012880000E0089500E008950091040208950A3CE2
:1012980043504D5F4469736B3E00001A000307001A
:1012A800F2003F00C00010000200028000051F018C
:1012B800FF07FF03FF0000010000002000051F01D9
:1012C800F907FF03FF0000010600DF93CF9310E149
:1012D800C1E5D4E0059109931A95E1F7CF91DF9123
:1012E800089509931FE0019109931A95E1F708956C
:1012F800A091EB01B091EC01000FA00FB71D08956C
:10130800F7DFDBCDA091EB01B091EC01109771F004
:1013180028E000E010E0DCDD2A95D9F70091EF0124
:101328001091F0010715170509F0D8DD0027089579
:1013380000270895C1E5D2E0E6E9F2E115910E949F
:10134800B80041F4E1E7F2E0C1E5D4E001E0C9DF2B
:101358000F6F089500270895E22F57DF0581168142
:10136800013000E4100751F4E1E5F2E010E00191EA
:10137800053E21F41A95D9F70F6F089500270895AF
:10138800E22F43DF05811681003000E41007A9F43D
:10139800C7ECD2E0E6E9F2E115910E94B80059F0F5
:1013A800E1E5F2E012E000240191053E31F40A94EF
:1013B800D9F71A95C9F70F6F0895002708952F9345
:1013C80000E010E09ED1B4DF71F4B4DF61F4D8DF3F
:1013D800E2ECF2E131F4C0DFE2EBF2E111F4E2EA2F
:1013E800F2E173DF0F6F2F910895E9DFD9F1E22F52
:1013F8000CDFC1E5D4E008810F701081107F012B4C
:101408000083098107830A81002331F41B811F703F
:10141800129510870F6F08950E9499000D0001E43E
:10142800020FF3DB0E9499003A20466F726D6174D7
:10143800206E6F7420737570706F727465643A20D3
:10144800546F6F206D75636820736563746F727372
:101458002070657220747261636B212000000E9405
:1014680099000D0000270895202FA9DF09F441C035
:1014780000E110E038DD09F43CC0D801E80100E0E3
:1014880010E026DD16960091ED011091EE0120DDA9
:101498000FE010E028DD59F1D801E2E5F4E0019110
:1014A8001ADDE136E1F71F978D01DE011A9610DD8E
:1014B80000915D0410915E040715170511F013DD06
:1014C800B1F006DD0091570410915804085F1F4FD2
:1014D80016950795169507951695079504DD39F025
:1014E800F7DC022F05DF8E01F3DC0F6F08958E0104
:1014F800F5DC0027089510811F701093FB011781F8
:101508001093FC01108512951F7000240394000CA1
:101518001A95E9F70092FD01089507FD25C006FD1B
:1015280037C004FD1EC005FD16C00E94990044493D
:10153800534B20492F4F3A20496E76616C696420DD
:1015480046756E6374696F6E20636F64653A200038
:101558000E94680040C67092F101F7987092FE01EF
:101568000895F69BF798089570920402F49AE09112
:10157800F4014BDE0081007F003009F408C0BBDFB6
:101588007092FE01F59A02E0009305025EC008958C
:1015980070920402F498E091F40137DE1081107F14
:1015A800103009F451C0A7DF037000930502023020
:1015B800A1F40091FD010093FE010091F401009354
:1015C800FF010091F501009300020091F6010093DC
:1015D80001020091F701009302020091FE0100232D
:1015E80079F10A950093FE010091F4011091FF0131
:1015F800011731F500910002109101022091F501C7
:101608003091F60102171307D9F40091F7011091F0
:1016180002020117A9F41395109302020090FC012D
:10162800101560F070920202009100021091010200
:101638000F5F1F4F0093000210930102F59805C039
:101648007092FE01F59A01C00895A091F701B0E0EB
:10165800C0E00091FB01A00FB71D2091F50130916A
:10166800F6010091FC01209FA00DB11D309FB00D27
:10167800C11D0A2F03700F9302E0C695B795A79571
:101688000A95D9F78D012091F40141D0E1E5F2E006
:1016980000E81F91109FE00DF11DA091F901B09194
:1016A800FA0120E8F49913C0F69AF894BBB928B85F
:1016B800ABB938B87AB848B800C0000009B168B802
:1016C80078946AB8019311962A9579F70DC001911B
:1016D800F894BBB928B8ABB938B80BB958B87894EE
:1016E80068B811962A9599F700910502013009F01A
:1016F800089500910402002309F008952CD0F6986B
:101708000895F59A04D00091040200230895709278
:1017180004020EB2F79A07FE14C0009006022015C4
:1017280039F400900702109008020015110591F095
:10173800F69B07C02F931F930F930DD00F911F9106
:101748002F91009307021093080220930602F5993F
:101758000ED0F6980895E091060257DD0081007FCB
:10176800003209F40FC3003109F403C10895E09170
:1017780006024BDD0081007F003209F418C30031F6
:1017880009F4FDC008957092F101C9E0D2E018E4AF
:1017980079921A95E9F739DC007031F4C0E0D0E0AD
:1017A800DE018EDC002311F000270895C9E0D2E0A5
:1017B80020E000914F04109150043AEA05351307D0
:1017C80079F023952093F10100E410E118837982E0
:1017D8007A827B827C827D820E8320E006DE1FC0B7
:1017E800EFE0F4E034E00481023539F4D3D02395F6
:1017F8002093F1012996283091F070963A9599F73F
:10180800EFE0F4E034E004810E3011F0063021F40A
:10181800E7D0F7D0DED003C070963A95A1F722271B
:101828000091F101201719F0E0DD2395F9CF00911F
:10183800F10100230895E9E0F2E0C091F101B1E47B
:1018480001811281238134810E9499000D000715BE
:1018580017052705370571F0A081A07FA03119F47D
:1018680027D02DD009C0A03219F422D035D004C019
:101878004BD002C01DD055D00E9434000E94990060
:101888002C2073697A653A2000000581168120E0D2
:1018980030E036952795179507950E9434000E94E9
:1018A80099004B422E003996B395CA9549F608958A
:1018B8000F930B2FAAD90AE3A8D90F9108950E9474
:1018C800990043502F4D20706172746974696F6E6E
:1018D8002061743A200008950E94990046415431CD
:1018E800362046696C652D496D6167652061743ADB
:1018F800200008950E94990052616D6469736B20FD
:1019080061743A20000008950E949900556E6B6E2C
:101918006F776E20456E7472792061743A200000EA
:1019280008950E949900417373756D696E6720432D
:10193800502F4D20696D6167652061743A20000061
:101948000895E091060261DC0091070210910802F7
:10195800A581B6810A171B0710F000270895A181F9
:10196800B281C381D481A00FB11FC71DD71D0F6FCE
:101978000895E7DF61F01CDC002349F405C0E1DFCE
:1019880031F09EDB002319F47092040208956092EE
:101998000402089500E108830085098301850A830C
:1019A80002850B8303850C8306851785012B29F493
:1019B80004850D8305850E8302C06D826E820895AD
:1019C80070926104C2E6D4E0799279927992799220
:1019D800089560927204609273046092710408958D
:1019E800CF93DF9360926104C2E6D4E00085099347
:1019F800018509930285099303850993DF91CF91A6
:101A08000895C0916104C03069F0C091F101C830F7
:101A180049F0E2E6F4E0A081B181C281D38150DBD4
:101A2800002311F000270895EEE5F2E0008100930D
:101A38006604E1E6F2E0008100937104E2E6F2E078
:101A4800019100936704108110936804E7E6F2E0BF
:101A5800019100937204108110937304EFE5F2E092
:101A680001911081E2E6F4E0A081B181C281D381C5
:101A7800A00FB11FC71DD71DA0936904B0936A04B6
:101A8800C0936B04D0936C04E9E6F4E0A081B181C3
:101A9800C281D38100917204109173042091710462
:101AA800271531F0A00FB11FC71DD71D2A95F8CFF4
:101AB800A0937504B0937604C0937704D093780408
:101AC800E0916704F0916804F695E795F695E79537
:101AD800F695E795F695E795A0917504B09176048B
:101AE800C0917704D0917804AE0FBF1FC71DD71DD2
:101AF800A0936D04B0936E04C0936F04D0937004E8
:101B080001E40093710400E00093740400916704F9
:101B1800009372040091680400937304A091750403
:101B2800B0917604C0917704D09178040091740440
:101B3800A00FB71DC71DD71DC3DA002311F000275A
:101B48000895E1E5F2E010E00081033469F50181D0
:101B5800003551F502810D3439F50381043421F53E
:101B68000481033509F505810B34F1F406810F353D
:101B7800D9F42091710407810217B1F40085093462
:101B880099F401850D3481F40285073469F4E093F2
:101B98007904F0937A0410937B0428C0E0917904C7
:101BA800F0917A0410917B04B0961395103109F0E6
:101BB800CBCF2091720430917304211B37092093F5
:101BC8007204309373042715370531F000917404BB
:101BD800039500937404A2CF0091710403950093B8
:101BE80071041AE501170CF48ECF2DC0C9E0D2E0BC
:101BF8002091F101222319F029962A95FBCF00E2C2
:101C08000883028D0983038D0A8300E00B830C830C
:101C1800048CA58DB68DE78D07101196E71DE69506
:101C2800B795A795A71DB71DE71DEE2311F0AFEFD8
:101C3800BFEFAD83BE830091F10103950093F101DD
:101C4800083009F0ABCF08950DD000916D04A00FB6
:101C580000916E04B01F00916F04C01F00917004C2
:101C6800D01F0895CC27DD271297009166040695AA
:101C7800002331F00695AA0FBB1FCC1FDD1FF8CF3C
:101C88000895E0910602C1DAC181D281A715B7058E
:101C9800E1F0AF93BF93FF27EC2FEE0FFF1F0D2F3F
:101CA800A0916904B0916A04C0916B04D0916C044E
:101CB800A00FB71DC71DD71D37DABF91AF91CE2F23
:101CC800DF2FE1E0AE1BB709E1CF0895E0910602EE
:101CD8009CDA0091070210910802A581B6810A17C3
:101CE8001B0710F000270895A02FB12FC72DD72D5F
:101CF800E0916604E695EE2331F0D695C795B79541
:101D0800A795E695F8CFCA2FE0916604E695EE23ED
:101D180019F0CC0FE695FBCFE02FEC1BE093740491
:101D2800C0917104D0910602CD1789F4C091720454
:101D3800D0917304CA1759F4DB1749F4A0917504BC
:101D4800B0917604C0917704D091780413C0C09103
:101D58000602C0937104A0937204B093730491DFD8
:101D6800DE0172DFA0937504B0937604C093770404
:101D7800D0937804E0917404AE0FB71DC71DD71D2A
:101D88000F6F0895A3DF81F013DA002351F00CC020
:101D9800FADC0F7749F09ADF39F00ADA002321F4E8
:101DA80000C07092040208956092040208958EDFC4
:101DB800D9F386D90023A9F3F7CFE5DC0F77A1F390
:101DC80085DF91F37DD9002379F708950895089563
:101DD80000014C0F510F0101E90509060201E9054F
:101DE80009060301330F300F04013E0F450F0D099B
:101DF8001A09150916014809910A400706041A0428
:101E080047071A0337034F015D0F5F0F0501E1060E
:101E18002A070603E406EA06800831073D070000A2
:101E2800689401C0E894DF93CF93E8EDFDE1059055
:101E38003591303081F0212F201910F0231710F040
:101E48003496F5CF0EF4329605901590F001099569
:101E5800CF91DF9108950FEFCF91DF91089500277B
:101E6800109129011711016010912C01103209F00D
:101E78000260089500271091290117110C94E905B3
:101E8800089510912C01103211F00C940906089550
:101E98000091290107110FEF08950E9499000D0084
:101EA8000E94990044656275673A20000E946800A4
:101EB800089500E0089500FB51F9089580E090E24C
:101EC800CCE7D4E0F09855270E9499000D000E94B5
:101ED80099004F6B2C205A38302D43505520697388
:101EE800206C6976652100000E9499000D00571149
:101EF80011C0F8949BB928B88BB938B87AB848B8E3
:101F080000C00000E9B168B878946AB80196F4E1B5
:101F18000995EDCF51FF06C0913020F09C3D10F49B
:101F28000E94C20050FF11C05A7F0E9499000D0004
:101F38000E949900427265616B20646574656374E0
:101F4800656421200000872D972DD3CF0895DC01EB
:101F58001197F894BBB928B8ABB938B87AB848B86B
:101F680000C0000069B168B878946AB8687370E016
:101F78000895642F792D08956981788108956B817A
:101F88007A8108956D817C810895B881A981F8943A
:101F9800BBB928B8ABB938B87AB848B800C000009F
:101FA80099B068B878946AB80895BA81AB81F89402
:101FB800BBB928B8ABB938B87AB848B800C000007F
:101FC80099B068B878946AB80895BC81AD81F894DE
:101FD800BBB928B8ABB938B87AB848B800C000005F
:101FE80069B168B878946AB80895D701F894BBB90C
:101FF80028B8ABB938B87AB848B800C0000069B199
:1020080068B878946AB81196F894BBB928B8ABB98F
:1020180038B87AB848B800C0000079B168B8789480
:102028006AB80895F8949BB928B88BB938B87AB8C3
:1020380048B800C0000069B168B878946AB80196D9
:102048000895F8949BB928B88BB938B87AB848B8C5
:1020580000C0000069B168B878946AB80196F8942D
:102068009BB928B88BB938B87AB848B800C000000E
:1020780079B168B878946AB801960895962E08954B
:1020880068830895698308956A8308956B83089522
:102098006C8308956D830895972E462F089578834D
:1020A800698308957A836B8308957C836D8308958B
:1020B800B881A981F894BBB928B8ABB938B89BB82E
:1020C80058B8789468B80895BA81AB81F894BBB9C8
:1020D80028B8ABB938B89BB858B8789468B8089598
:1020E800BC81AD81F894BBB928B8ABB938B86BB925
:1020F80058B8789468B80895D701F894BBB928B847
:10210800ABB938B86BB958B8789468B81196F894E0
:10211800BBB928B8ABB938B87BB958B8789468B89F
:1021280008957B010895CB010895772766230AF463
:102138007095860F971F0895D701F894BBB928B8F2
:10214800ABB938B87AB848B800C0000089B168B8E7
:1021580078946AB81196F894BBB928B8ABB938B86E
:102168007AB848B800C0000099B168B878946AB8DD
:1021780011967D010895D7011197F894BBB928B835
:10218800ABB938B89BB958B8789468B81197F8942F
:10219800BBB928B8ABB938B88BB958B8789468B80F
:1021A8007D01CB010895F8947BB928B86BB938B88C
:1021B8009BB858B8789468B8089501970E94C200EF
:1021C8000E949900496E76616C6964206F70636F34
:1021D800646521200000FFCF019752FD08955460E7
:1021E8000E94C2000E9499004350552068616C7497
:1021F8006564212000000895092D162F11DE089529
:10220800162F10DE902E0895417001E0600F0FB771
:1022180002FB47F901FB46F905FB44F903FB42F9C8
:102228000895417001E0900E0FB702FB47F901FBDA
:1022380046F905FB44F903FB42F9089561500FB7CD
:1022480002FB47F901FB46F905FB44F903FB42F998
:102258004260089501E0901A0FB702FB47F901FBAD
:1022680046F905FB44F903FB42F9426008956F5FA4
:102278007F4F08956150704008954C7E990C18F472
:1022880001E0902A416008954C7E969418F400E885
:10229800902A41600895889440FD08944C7E90FAF5
:1022A80040F997940895889440FD08944C7E97FAD5
:1022B80040F9991C0895960E0FB7F6E4E92D44915C
:1022C80000FB40F905FB44F903FB42F908958894A3
:1022D80040FD0894961E0FB7F6E4E92D449100FBE3
:1022E80040F905FB44F903FB42F90895961A0FB724
:1022F800F6E4E92D449100FB40F905FB44F903FBA2
:1023080042F942600895192D161B0FB7F6E4E12F24
:10231800449100FB40F905FB44F903FB42F9426094
:102328000895889440FD0894960A0FB7F6E4E92DBD
:10233800449100FB40F905FB44F903FB42F9426074
:1023480008959622F6E4E92D449140610895962A6D
:10235800F6E4E92D449108959626F6E4E92D449192
:1023680008950D811C81600F711F6D837C830FB7E9
:1023780000FB40F905FB44F94D7F0895DB010D8111
:10238800F894BBB928B8ABB938B80BB958B8789431
:1023980068B811960C81F894BBB928B8ABB938B8AD
:1023A8000BB958B8789468B80895DB01F894BBB9AC
:1023B80028B8ABB938B87AB848B800C0000069B1D5
:1023C80068B878946AB81196F894BBB928B8ABB9CC
:1023D80038B87AB848B800C0000079B168B87894BD
:1023E8006AB80895F8947BB928B86BB938B87AB840
:1023F80048B800C0000069B168B878946AB8089510
:1024080070E041FD21C010E0062F0F700A3048F03F
:102418007660106140FD02C0603910F0706611608E
:102428000DC040FD02C0603A10F07066116044FFB4
:1024380005C07660062F0F70063000F4670FF6E4CB
:10244800E62F4491412B089512E0062F0F700A30B1
:1024580040F0766040FD02C0603910F0706611608F
:102468000EC040FD02C0603A10F07066116044FF73
:1024780006C07660062F0F70063008F41061671BDF
:10248800F6E4E62F4491412B08954D7E416008956E
:102498004D7F40FB44F901E0402708959094426144
:1024A8000895D7011197F894BBB928B8ABB938B8D3
:1024B8007BB958B8789468B81197F894BBB928B81C
:1024C800ABB938B86BB958B8789468B87D01089535
:1024D800D701F894BBB928B8ABB938B87AB848B8B6
:1024E80000C0000069B168B878946AB81196F89489
:1024F800BBB928B8ABB938B87AB848B800C000003A
:1025080079B168B878946AB811967D0108950D81FB
:102518001C816D837C83B80108950C89037F0C8B23
:1025280008950C890C600C8B089546FF08950F914F
:102538000F91089546FD08950F910F91089540FF5A
:1025480008950F910F91089540FD08950F910F91EF
:10255800089542FF08950F910F91089542FD08953F
:102568000F910F91089547FF08950F910F910895C6
:1025780047FD08950F910F91089508810A950883E2
:1025880029F0605880589709860F971D08950C8583
:102598001D854C879D86402F912E0895ECE7F4E029
:1025A80026E000811681068311932A95D1F70895B4
:1025B800F8949BB928B88BB938B87AB848B800C02D
:1025C8000000E9B168B878946AB80196F2E2099413
:1025D800F198F8949BB928B88BB938B87AB848B844
:1025E80000C00000E9B168B878946AB80196F8E1CB
:1025F8000994F19AF8949BB928B88BB938B87AB885
:1026080048B800C00000E9B168B878946AB8019683
:10261800F8E10994F8949BB928B88BB938B87AB816
:1026280048B800C00000E9B168B878946AB8019663
:10263800FAE10994F19903C0BE85AF8502C0B88953
:10264800A989F8949BB928B88BB938B87AB848B82A
:1026580000C0000009B168B878946AB801961127DB
:1026680000230AF41095A00FB11FF894BBB928B83D
:10267800ABB938B87AB848B800C0000069B168B8D2
:1026880078946AB8F8949BB928B88BB938B87AB8EE
:1026980048B800C00000E9B168B878946AB80196F3
:1026A800FEE10995F894BBB928B8ABB938B86BB94D
:0826B80058B8789468B8089541
:0428000008955ECF0A
:0426C000C4DCF1CCB9
:0428040059CC5ECF7E
:0626C4005DDCD7DDEECC69
:0228080060CF9F
:0626CA006881A1DDDCCCFB
:02280A0062CF9B
:0626D0006881B8DDD9CCE1
:02280C0064CF97
:0426D600AADCD7CCD7
:06280E0039CDC2CE63CFFC
:0426DA0052DC46CEBA
:04281400BECB63CF05
:0626DE0050DCCDDDE1CC73
:0228180065CF8A
:0626E400698194DDD1CCF8
:02281A0067CF86
:0626EA006981ABDDCECCDE
:02281C0069CF82
:0426F0009DDCCCCCD5
:04281E0038CD69CF79
:0426F4009BDC45CF57
:022822006ACF7B
:0426F800A8DCD8CCB6
:0428240055CC6ACF56
:0626FC0044DCBBDDD5CC7F
:022828006CCF73
:062702006A8185DDC4CCF4
:02282A006ECF6F
:062708006A819CDDC1CCDA
:02282C0070CF6B
:04270E008EDCBFCCD2
:04282E003FCD70CF5B
:042712008CDC0ECD80
:0228320071CF64
:0427160037DC28CEB6
:04283400BECB71CFD7
:06271A0035DCAFDDC6CC8A
:0228380073CF5C
:062720006B8176DDB7CCF1
:02283A0075CF58
:062726006B818DDDB4CCD7
:02283C0077CF54
:04272C007FDCB2CCD0
:04283E002FCD77CF54
:062730007DDCFFDEFECCA3
:0228420079CF4C
:0427360089DCBCCCB2
:022844007ACF49
:04273A0087DC23CE47
:022846007BCF46
:06273E0026DC9ADDB7CC99
:022848007DCF42
:062744006C8164DDA7CCEE
:02284A007FCF3E
:06274A006C817BDDA4CCD4
:02284C0081CF3A
:042750006DDCA2CCCE
:02284E0082CF37
:06275400692D58DE95CC52
:0228500084CF33
:06275A0068DCEFDEE9CCB3
:0228520086CF2F
:0427600015DC03CEB3
:0228540087CF2C
:0627640072DC25DEA4CCAE
:0228560089CF28
:06276A0010DC87DDA1CCAC
:022858008BCF24
:062770006D814EDD93CCEB
:02285A008DCF20
:062776006D8165DD90CCD1
:02285C008FCF1C
:04277C0057DC8ECCCC
:04285E0022CE8FCF28
:0627800055DCE1DED6CCC1
:0228620091CF14
:0427860061DCD0CC76
:0228640092CF11
:04278A005FDC10CD33
:0228660093CF0E
:06278E00B70172DDCBCCA7
:0228680095CF0A
:062794001EDC3CDDA7CCB9
:02286A0097CF06
:06279A001BDC53DDA4CCA2
:02286C0099CF02
:0427A00045DCA2CCA6
:04286E0011CE99CF1F
:0627A40043DCD4DEC4CCCE
:022872009BCFFA
:0427AA00B701DECDC8
:022874009CCFF7
:0627AE004DDC1DDE68CCCD
:022876009ECFF3
:0627B400B70162DDB8CCA4
:06287800D8CCF0CC9ECF8D
:0427BA0038DC63CCD8
:06287E000CCE08959DCF71
:0427BE00698163CCFE
:022884009ECFE5
:0427C2006A8161CCFB
:022886009FCFE2
:0427C6006B815FCCF8
:02288800A0CFDF
:0427CA006C815DCCF5
:02288A00A1CFDC
:0427CE006D815BCCF2
:02288C00A2CFD9
:0427D200FFDB59CC04
:02288E00A3CFD6
:0427D600692D57CC46
:02289000A4CFD3
:0427DA00688157CCEF
:042892000895A4CF32
:0427DE006A8155CCEB
:02289600A5CFCC
:0427E2006B8153CCE8
:02289800A6CFC9
:0427E6006C8151CCE5
:02289A00A7CFC6
:0427EA006D814FCCE2
:02289C00A8CFC3
:0427EE00F1DB4DCC02
:02289E00A9CFC0
:0427F200692D4BCC36
:0228A000AACFBD
:0427F60068814BCCDF
:0228A200AEC0C6
:042A0000698146CBD7
:0428A4000895AEC025
:042A04006B8144CBD3
:0228A800AFC0BF
:042A08006C8142CBD0
:0228AA00B0C0BC
:042A0C006D8140CBCD
:0228AC00B1C0B9
:042A1000E0DA3ECBFF
:0228AE00B2C0B6
:042A1400692D3CCB21
:0228B000B3C0B3
:042A180068813CCBCA
:0228B200B4C0B0
:042A1C0069813ACBC7
:0228B400B5C0AD
:042A20006A8138CBC4
:0428B6000895B5C00C
:042A24006C8136CBC0
:0228BA00B6C0A6
:042A28006D8134CBBD
:0228BC00B7C0A3
:042A2C00D2DA32CBFD
:0228BE00B8C0A0
:042A3000692D30CB11
:0228C000B9C09D
:042A3400688130CBBA
:0228C200BAC09A
:042A380069812ECBB7
:0228C400BBC097
:042A3C006A812CCBB4
:0228C600BCC094
:042A40006B812ACBB1
:0428C8000895BCC0F3
:042A44006D8128CBAD
:0228CC00BDC08D
:042A4800C4DA26CBFB
:0228CE00BEC08A
:042A4C00692D24CB01
:0228D000BFC087
:042A5000688124CBAA
:0228D200C0C084
:042A5400698122CBA7
:0228D400C1C081
:042A58006A8120CBA4
:0228D600C2C07E
:042A5C006B811ECBA1
:0228D800C3C07B
:042A60006C811CCB9E
:0428DA000895C3C0DA
:042A6400B6DA1ACBF9
:0228DE00C4C074
:042A6800692D18CBF1
:0228E000C5C071
:042A6C0068813CCB76
:0228E200C6C06E
:042A700069813ACB73
:0228E400C7C06B
:042A74006A8138CB70
:0228E600C8C068
:042A78006B8136CB6D
:0228E800C9C065
:042A7C006C8134CB6A
:0228EA00CAC062
:042A80006D8132CB67
:0428EC0079CCCAC019
:042A8400692D30CBBD
:0228F000CBC05B
:042A88006881FCCA9B
:0228F200CCC058
:042A8C006981FACA98
:0228F400CDC055
:042A90006A81F8CA95
:0228F600CEC052
:042A94006B81F6CA92
:0228F800CFC04F
:042A98006C81F4CA8F
:0228FA00D0C04C
:042A9C006D81F2CA8C
:0228FC00D1C049
:042AA00098DAF0CA06
:0428FE000895D1C0A8
:042AA40068810BCC6E
:02290200D2C041
:042AA800698109CC6B
:02290400D3C03E
:042AAC006A8107CC68
:02290600D4C03B
:042AB0006B8105CC65
:02290800D5C038
:042AB4006C8103CC62
:02290A00D6C035
:042AB8006D8101CC5F
:02290C00D7C032
:042ABC008ADAFFCBE8
:02290E00D8C02F
:042AC000692DFDCBB4
:02291000D9C02C
:042AC400688107CC52
:02291200DAC029
:042AC800698105CC4F
:02291400DBC026
:042ACC006A8103CC4C
:02291600DCC023
:042AD0006B8101CC49
:02291800DDC020
:042AD4006C81FFCB47
:02291A00DEC01D
:042AD8006D81FDCB44
:02291C00DFC01A
:042ADC007ADAFBCBDC
:02291E00E0C017
:042AE000692DF9CB98
:02292000E1C014
:042AE400688106CC33
:02292200E2C011
:042AE800698104CC30
:02292400E3C00E
:042AEC006A8102CC2D
:02292600E4C00B
:042AF0006B8100CC2A
:02292800E5C008
:042AF4006C81FECB28
:02292A00E6C005
:042AF8006D81FCCB25
:02292C00E7C002
:042AFC006ADAFACBCD
:02292E00E8C0FF
:042B0000692DF8CB78
:02293000E9C0FC
:042B0400688111CC07
:02293200EAC0F9
:042B080069810FCC04
:02293400EBC0F6
:042B0C006A810DCC01
:02293600ECC0F3
:042B10006B810BCCFE
:02293800EDC0F0
:042B14006C8109CCFB
:02293A00EEC0ED
:042B18006D8107CCF8
:02293C00EFC0EA
:042B1C005ADA05CCB0
:02293E00F0C0E7
:042B2000692D03CC4C
:02294000F1C0E4
:042B2400688111CCE7
:02294200F2C0E1
:042B280069810FCCE4
:02294400F3C0DE
:042B2C006A810DCCE1
:02294600F4C0DB
:042B30006B810BCCDE
:02294800F5C0D8
:042B34006C8109CCDB
:02294A00F6C0D5
:042B38006D8107CCD8
:02294C00F7C0D2
:042B3C004ADA05CCA0
:02294E00F8C0CF
:042B4000692D03CC2C
:02295000F9C0CC
:042B440068810CCCCC
:02295200FAC0C9
:042B480069810ACCC9
:02295400FBC0C6
:042B4C006A8108CCC6
:02295600FCC0C3
:042B50006B8106CCC3
:02295800FDC0C0
:042B54006C8104CCC0
:02295A00FEC0BD
:042B58006D8102CCBD
:02295C00FFC0BA
:042B5C003ADA00CC95
:02295E0000C1B6
:042B6000692DFECB12
:0229600001C1B3
:042B64006881F7CBC2
:0229620002C1B0
:042B68006981F5CBBF
:0229640003C1AD
:042B6C006A81F3CBBC
:0229660004C1AA
:042B70006B81F1CBB9
:0229680005C1A7
:042B74006C81EFCBB6
:02296A0006C1A4
:042B78006D81EDCBB3
:02296C0007C1A1
:042B7C002ADAEBCB9B
:02296E0008C19E
:042B8000692DE9CB07
:0229700009C19B
:042B84006881C3CBD6
:022972000AC198
:042B88006981C1CBD3
:022974000BC195
:042B8C006A81BFCBD0
:022976000CC192
:042B90006B81BDCBCD
:022978000DC18F
:042B94006C81BBCBCA
:02297A000EC18C
:042B98006D81B9CBC7
:02297C000FC189
:042B9C001ADAB7CBBF
:02297E0010C186
:042BA000692DB5CB1B
:0229800011C183
:042BA400C6DCCCCAF5
:0229820012C180
:042BA80097DC7DCA6F
:0229840013C17D
:062BAC004EDAC1DCBECAD6
:0229860015C179
:042BB2004BDABCCA74
:0229880016C176
:062BB60049DABCDCE1CAB3
:02298A0018C172
:042BBC00E1D975CC1A
:02298C0019C16F
:042BC00035DA7DCBBA
:02298E001AC16C
:042BC400C8D9DBCAC7
:022990001BC169
:042BC800B9DCBACAF0
:04299200D6CB1BC1C4
:062BCC003EDAB6DCAECAE1
:0429960042CE1CC150
:062BD2003BDAB3DCD3CABC
:02299A001EC15C
:042BD80038DAD1CA4C
:02299C001FC159
:042BDC0027DA7BCBAE
:04299E0012C11FC182
:042BE000B2DCAECAEB
:0229A20020C152
:042BE40079DC62CA6C
:0229A40021C14F
:062BE80030DAADDCA0CAEA
:0229A60023C14B
:042BEE001EDA07CB19
:0229A80024C148
:062BF2002BDAA8DCC3CAC7
:0229AA0026C144
:042BF800C6D957CC17
:0229AC0027C141
:042BFC0017DA7ACB9F
:0429AE000AC127C172
:042C0000A7DC9ECAE5
:0429B200F8CD27C174
:062C040022DAA4DC92CAF2
:0229B60029C135
:042C0A0010DAFDCA15
:0229B8002AC132
:062C0E001DDA9FDCB5CACF
:0429BA000ECE2BC151
:042C14000BDA89CB83
:0429BE0002C12BC166
:042C1800A0DC92CAE0
:0229C2002CC126
:042C1C005DDC49CA68
:0229C4002DC123
:062C200014DA9BDC84CAFB
:0229C6002FC11F
:062C2600E5D976DC6ACA64
:0229C80031C11B
:062C2C000EDA95DCA6CAD9
:0229CA0033C117
:042C3200ACD93ACC13
:0229CC0034C114
:042C3600FAD988CB74
:0429CE00FAC034C156
:042C3A0094DC81CADB
:0229D20035C10D
:042C3E00A6D976CAD3
:0229D40036C10A
:062C420003DA8FDC73CA07
:0229D60038C106
:062C48009ED965DC2FCAD5
:0229D8003AC102
:062C4E00FDD989DC95CAE6
:0429DA00EECD3BC142
:042C5400EBD984CB69
:0429DE00F2C03BC147
:042C58008ADC72CAD6
:0229E2003CC1F6
:042C5C003DDC20CA71
:0229E4003DC1F3
:062C6000F4D985DC64CA12
:0429E6009DCD3EC184
:062C6600F1D982DC89CAED
:0229EA0040C1EA
:042C6C0086D91DCC1C
:0229EC0041C1E7
:042C7000DDD971CB6E
:0429EE00EAC041C139
:042C740081DC64CAD1
:0229F20042C1E0
:042C780089D957CAD5
:0229F40043C1DD
:062C7C00E6D97CDC56CA1B
:0429F60099CD44C172
:062C8200E3D979DC7BCAF6
:0429FA00FFCD45C107
:042C8800D1D941CB92
:0229FE00E2C035
:102C8C0001970895DC011196F894BBB928B8ABB93B
:102C9C0038B87AB848B800C0000069B168B8789400
:102CAC006AB80895F19B6E85F19968890895F19B36
:102CBC006F85F19969890895F19903C0BE85AF8537
:102CCC0002C0B889A989F8949BB928B88BB938B8CF
:102CDC007AB848B800C0000069B168B878946AB88E
:102CEC000196772766230AF47095A60FB71FF89400
:102CFC00BBB928B8ABB938B87AB848B800C000002E
:102D0C0069B168B878946AB80895F19903C06F8571
:102D1C007E850895698978890895F19B6E87F1996C
:102D2C00688B0895F19B6F87F199698B0895F199E0
:102D3C0003C0BE85AF8502C0B889A989F8949BB938
:102D4C0028B88BB938B87AB848B800C0000009B1B7
:102D5C0068B878946AB80196112700230AF4109584
:102D6C00A00FB11FF894BBB928B8ABB938B86BB980
:102D7C0058B8789468B80895F894BBB928B8ABB92A
:102D8C0038B86BB958B8789468B80895F19903C0FD
:102D9C00BE85AF8502C0B889A989F8949BB928B8BB
:102DAC008BB938B87AB848B800C0000009B168B817
:102DBC0078946AB801960196112700230AF41095AD
:102DCC00A00FB11FF894BBB928B8ABB938B86BB920
:102DDC0058B8789468B80895F19903C06F877E87C6
:102DEC000895698B788B0895DB01F19B0F85F19920
:102DFC000989F894BBB928B8ABB938B80BB958B82D
:102E0C00789468B81196F19B0E85F1990889F8941D
:102E1C00BBB928B8ABB938B80BB958B8789468B8FE
:102E2C000895F19905C00F851E856F877E8704C0B4
:102E3C0009891889698B788BB8010895F19907C0B5
:102E4C000F851E85600F711F6F877E8706C00989ED
:102E5C001889600F711F698B788B0FB700FB40F9D5
:082E6C0005FB44F94D7F0895B8
:1030000045CE44CE43CE42CE41CE40CE3FCE3ECE44
:043010003DCE30CFB2
:042E740085D8E8CF46
:103014003BCE3ACE39CE38CE37CE36CE35CE34CE80
:1030240033CE32CE31CE30CE2FCE2ECE2DCE22CFB9
:042E780086D8E6CF43
:103034002BCE2ACE29CE28CE27CE26CE25CE1CCFE7
:042E7C00E6D8B2CF13
:023044001DCF9E
:042E8000E4D8B8CF0B
:023046001ECF9B
:062E840048DFF7D9ADCFD5
:0230480020CF97
:062E8A0012DFC1D94BCF9D
:02304A0022CF93
:062E90000FDFD8D948CF86
:02304C0024CF8F
:042E9600CAD846CF81
:06304E001ECE1DCE23CFB3
:042E9A003DDFD5CF74
:0230540024CF87
:062E9E00D5D888DAA0CFB0
:0230560026CF83
:062EA40038DFEAD99DCFE2
:0230580028CF7F
:062EAA0007DFB1D940CFA3
:02305A002ACF7B
:062EB00004DFC8D93DCF8C
:02305C002CCF77
:042EB600BAD83BCF7C
:0C305E0016CE15CE14CE13CE12CE28CF05
:062EBA0004DFA9D962CF7C
:02306A002ACF6B
:062EC00001DFC0D95FCF65
:02306C002CCF67
:042EC600E4DE67CF10
:06306E000ECE0DCE2BCFAB
:042ECA00B701BDCFC0
:103074000BCE0ACE09CE08CE07CE06CE05CE04CEA0
:0630840003CE02CE22CFB4
:042ECE00F0DEDBC88F
:02308A0023CF52
:042ED200F3DED9C88A
:02308C0024CF4F
:042ED600F6DED7C885
:0C308E00FECDFDCDFCCDFBCDFACD20CF5A
:042EDA00EADED7C88D
:02309A0021CF44
:042EDE00EDDED5C888
:02309C0022CF41
:042EE200F0DED3C883
:0C309E00F6CDF5CDF4CDF3CDF2CD1ECF74
:042EE600E4DED3C88B
:0230AA001FCF36
:042EEA00E7DED1C886
:0230AC0020CF33
:042EEE00EADECFC881
:0C30AE00EECDEDCDECCDEBCDEACD1CCF8E
:042EF200DEDECFC889
:0230BA001DCF28
:042EF600E1DECDC884
:0230BC001ECF25
:042EFA00E4DECBC87F
:0430BE00E6CD1ECF6E
:042EFE00688112CF06
:0230C2001FCF1E
:042F0200698110CF02
:0230C40020CF1B
:042F06006A810ECFFF
:0230C60021CF18
:042F0A006B810CCFFC
:0430C800E1CD21CF66
:042F0E00D5DE0ACF33
:0230CC0022CF11
:042F1200D8DEC1C87C
:0230CE0023CF0E
:042F1600692D06CF4C
:0230D00024CF0B
:042F1A00688109CFF2
:0230D20025CF08
:042F1E00698107CFEF
:0230D40026CF05
:042F22006A8105CFEC
:0230D60027CF02
:042F26006B8103CFE9
:0230D80028CFFF
:042F2A00C2DE01CF33
:0430DA00D8CD28CF56
:042F2E00CADEB5C87A
:0230DE0029CFF8
:042F3200692DFDCE3A
:0230E0002ACFF5
:042F3600688100CFDF
:0230E2002BCFF2
:042F3A006981FECEDD
:0230E4002CCFEF
:042F3E006A81FCCEDA
:0230E6002DCFEC
:042F42006B81FACED7
:0230E8002ECFE9
:042F46006C81F8CED4
:0230EA002FCFE6
:042F4A006D81F6CED1
:0430EC00CFCD2FCF46
:042F4E00692DF4CE27
:0A30F000CDCDCCCDCBCDCACD2CCF79
:042F5200AEDE97C890
:0230FA002DCFD8
:042F5600B1DE95C88B
:0230FC002ECFD5
:042F5A00B4DE93C886
:0C30FE00C6CDC5CDC4CDC3CDC2CD2ACFF8
:042F5E00A8DEAEC972
:02310A002BCFC9
:042F6200ABDEACC96D
:02310C002CCFC6
:042F6600AEDEAAC968
:0C310E00BECDBDCDBCCDBBCDBACD28CF11
:042F6A00A2DEB4C966
:02311A0029CFBB
:042F6E00A5DEB2C961
:02311C002ACFB8
:042F7200A8DEB0C95C
:0C311E00B6CDB5CDB4CDB3CDB2CD26CF2B
:042F76009CDEBDC957
:02312A0027CFAD
:042F7A009FDEBBC952
:02312C0028CFAA
:042F7E00A2DEB9C94D
:0C312E00AECDADCDACCDABCDAACD24CF45
:042F820096DED2C93C
:02313A0025CF9F
:042F860099DED0C937
:02313C0026CF9C
:042F8A009CDECEC932
:0C313E00A6CDA5CDA4CDA3CDA2CD22CF5F
:042F8E0090DEDCC92C
:02314A0023CF91
:042F920093DEDAC927
:02314C0024CF8E
:042F960096DED8C922
:0C314E009ECD9DCD9CCD9BCD9ACD20CF79
:042F9A008ADEE1C921
:02315A0021CF83
:042F9E008DDEDFC91C
:02315C0022CF80
:042FA20090DEDDC917
:0C315E0096CD95CD94CD93CD92CD1ECF93
:042FA60084DED6C926
:02316A001FCF75
:042FAA0087DED4C921
:02316C0020CF72
:042FAE008ADED2C91C
:0C316E008ECD8DCD8CCD8BCD8ACD1CCFAD
:042FB2007EDEACC94A
:02317A001DCF67
:042FB60081DEAAC945
:02317C001ECF64
:042FBA0084DEA8C940
:10317E0086CD85CD84CD83CD82CD81CD80CD7FCDC5
:10318E007ECD7DCD7CCD7BCD52CA79CD78CD77CD20
:10319E0076CD75CD74CD73CD72CD71CD70CD6FCD25
:1031AE006ECD6DCD6CCD6BCD6ACD69CD68CD67CD55
:0631BE0066CD65CDFDCEDB
:042FBE008CDA11CFC9
:0431C40063CDFDCE0C
:062FC20017D834DF9CC8A3
:0431C80061CDFECE09
:042FC800A6DE6FCA48
:0831CC005FCD5ECD5DCDFCCEB0
:042FCC00A4DEAFC808
:1031D4005BCD5ACD59CD58CD57CD56CD55CD54CDC7
:1031E40053CD52CD51CD50CD4FCD4ECD4DCDEECE54
:042FD000A2DEABC80A
:0C31F4004BCD4ACD49CD48CD47CD46CD4E
:102FD4000027660F071D602BF6E4E62F4491402B73
:102FE4000895669508F46068F6E4E62F449167FB5B
:042FF40040F9089503
:10320000889440FD0894661F0FB7F6E4E62F4491BA
:1032100000FB40F9089567950FB740FB67F9F6E4A6
:10322000E62F449100FB40F90895660F0FB7F6E4CE
:10323000E62F449100FB40F9089566950FB766FBB1
:1032400067F9F6E4E62F449100FB40F908950894ED
:10325000661F0FB7F6E4E62F449100FB40F908958E
:1032600066950FB7F6E4E62F449100FB40F9089508
:1032700000E80DC000E40BC000E209C000E107C097
:1032800008E005C004E003C002E001C001E006233D
:103290000FB740614D7F01FB46F90895688308959B
:1032A000698308956A8308956B8308956C830895F4
:1032B0006D830895962E0895BC81AD81F894BBB9B5
:1032C00028B8ABB938B87AB848B800C0000069B1BE
:0832D00068B878946AB808950B
:023400006BCF90
:0632D80068817CDEDFCFFF
:023402006DCF8C
:0632DE00698179DEDECFFC
:023404006FCF88
:0632E4006A8176DEDDCFF9
:0234060071CF84
:0632EA006B8173DEDCCFF6
:0234080073CF80
:0632F0006C8170DEDBCFF3
:02340A0075CF7C
:0632F6006D816DDEDACFF0
:02340C0077CF78
:0832FC00DDDF6ADE0C947410A2
:02340E007ACF73
:06330400692D66DED5CF45
:023410007CCF6F
:06330A0068816CDEC6CFF5
:023412007ECF6B
:06331000698169DEC5CFF2
:0234140080CF67
:063316006A8166DEC4CFEF
:0234160082CF63
:06331C006B8163DEC3CFEC
:0234180084CF5F
:063322006C8160DEC2CFE9
:02341A0086CF5B
:063328006D815DDEC1CFE6
:02341C0088CF57
:08332E00C4DF5ADE0C94741098
:02341E008BCF52
:06333600692D56DEBCCF3C
:023420008DCF4E
:06333C00688160DFADCFE7
:023422008FCF4A
:0633420069815DDFACCFE4
:0234240091CF46
:063348006A815ADFABCFE1
:0234260093CF42
:06334E006B8157DFAACFDE
:0234280095CF3E
:063354006C8154DFA9CFDB
:02342A0097CF3A
:06335A006D8151DFA8CFD8
:02342C0099CF36
:08336000ABDF4EDF0C9474108A
:02342E009CCF31
:06336800692D4ADFA3CF2E
:023430009ECF2D
:06336E00688152DF94CFDC
:02343200A0CF29
:0633740069814FDF93CFD9
:02343400A2CF25
:06337A006A814CDF92CFD6
:02343600A4CF21
:063380006B8149DF91CFD3
:02343800A6CF1D
:063386006C8146DF90CFD0
:02343A00A8CF19
:06338C006D8143DF8FCFCD
:02343C00AACF15
:0833920092DF40DF0C9474107F
:02343E00ADCF10
:06339A00692D3CDF8ACF23
:02344000AFCF0C
:0633A000688143DF7BCFD2
:02344200B1CF08
:0633A600698140DF7ACFCF
:02344400B3CF04
:0633AC006A813DDF79CFCC
:02344600B5CF00
:0633B2006B813ADF78CFC9
:02344800B7CFFC
:0633B8006C8137DF77CFC6
:02344A00B9CFF8
:0633BE006D8134DF76CFC3
:02344C00BBCFF4
:0833C40079DF31DF0C94741075
:02344E00BECFEF
:0633CC00692D2DDF71CF19
:02345000C0CFEB
:0633D200688132DF62CFCA
:02345200C2CFE7
:0633D80069812FDF61CFC7
:02345400C4CFE3
:0633DE006A812CDF60CFC4
:02345600C6CFDF
:0633E4006B8129DF5FCFC1
:02345800C8CFDB
:0633EA006C8126DF5ECFBE
:02345A00CACFD7
:0633F0006D8123DF5DCFBB
:02345C00D1C0DD
:083600005BDE1BDE0C9474106C
:02345E00D4C0D8
:06360800692D17DE53CE10
:02346000D6C0D4
:06360E0068811EDE44CEBF
:02346200D8C0D0
:0636140069811BDE43CEBC
:02346400DAC0CC
:06361A006A8118DE42CEB9
:02346600DCC0C8
:063620006B8115DE41CEB6
:02346800DEC0C4
:063626006C8112DE40CEB3
:02346A00E0C0C0
:06362C006D810FDE3FCEB0
:02346C00E2C0BC
:0836320042DE0CDE0C94741062
:02346E00E5C0B7
:06363A00692D08DE3ACE06
:02347000E7C0B3
:0636400068810EDE2BCEB6
:02347200E9C0AF
:0636460069810BDE2ACEB3
:02347400EBC0AB
:06364C006A8108DE29CEB0
:02347600EDC0A7
:063652006B8105DE28CEAD
:02347800EFC0A3
:063658006C8102DE27CEAA
:02347A00F1C09F
:06365E006D81FFDD26CEA8
:02347C00F3C09B
:0836640029DEFCDD0C9474105A
:02347E00F6C096
:06366C00692DF8DD21CEFE
:02348000F8C092
:0436720068810BCE92
:02348200F9C08F
:04367600698109CE8F
:02348400FAC08C
:04367A006A8107CE8C
:02348600FBC089
:04367E006B8105CE89
:02348800FCC086
:043682006C8103CE86
:02348A00FDC083
:043686006D8101CE83
:02348C00FEC080
:04368A0016DEFFCD7C
:02348E00FFC07D
:04368E00692DFDCDD8
:0234900000C179
:043692006881F9CD85
:0234920001C176
:043696006981F7CD82
:0234940002C173
:04369A006A81F5CD7F
:0234960003C170
:04369E006B81F3CD7C
:0234980004C16D
:0436A2006C81F1CD79
:02349A0005C16A
:0436A6006D81EFCD76
:02349C0006C167
:0436AA0006DEEDCD7E
:02349E0007C164
:0436AE00692DEBCDCA
:0234A00008C161
:0436B2006881E7CD77
:0234A20009C15E
:0436B6006981E5CD74
:0234A4000AC15B
:0436BA006A81E3CD71
:0234A6000BC158
:0436BE006B81E1CD6E
:0234A8000CC155
:0436C2006C81DFCD6B
:0234AA000DC152
:0436C6006D81DDCD68
:0234AC000EC14F
:0436CA00F6DDDBCD81
:0234AE000FC14C
:0436CE00692DD9CDBC
:0234B00010C149
:0436D2006881D5CD69
:0234B20011C146
:0436D6006981D3CD66
:0234B40012C143
:0436DA006A81D1CD63
:0234B60013C140
:0436DE006B81CFCD60
:0234B80014C13D
:0436E2006C81CDCD5D
:0234BA0015C13A
:0436E6006D81CBCD5A
:0234BC0016C137
:0436EA00E6DDC9CD83
:0234BE0017C134
:0436EE00692DC7CDAE
:0234C00018C131
:0436F2006881C3CD5B
:0234C20019C12E
:0436F6006981C1CD58
:0234C4001AC12B
:0436FA006A81BFCD55
:0234C6001BC128
:0436FE006B81BDCD52
:0234C8001CC125
:043702006C81BBCD4E
:0234CA001DC122
:043706006D81B9CD4B
:0234CC001EC11F
:04370A00D6DDB7CD84
:0234CE001FC11C
:04370E00692DB5CD9F
:0234D00020C119
:043712006881B1CD4C
:0234D20021C116
:043716006981AFCD49
:0234D40022C113
:04371A006A81ADCD46
:0234D60023C110
:04371E006B81ABCD43
:0234D80024C10D
:043722006C81A9CD40
:0234DA0025C10A
:043726006D81A7CD3D
:0234DC0026C107
:04372A00C6DDA5CD86
:0234DE0027C104
:04372E00692DA3CD91
:0234E00028C101
:0437320068819FCD3E
:0234E20029C1FE
:0437360069819DCD3B
:0234E4002AC1FB
:04373A006A819BCD38
:0234E6002BC1F8
:04373E006B8199CD35
:0234E8002CC1F5
:043742006C8197CD32
:0234EA002DC1F2
:043746006D8195CD2F
:0234EC002EC1EF
:04374A00B6DD93CD88
:0234EE002FC1EC
:04374E00692D91CD83
:0234F00030C1E9
:0437520068818DCD30
:0234F20031C1E6
:0437560069818BCD2D
:0234F40032C1E3
:04375A006A8189CD2A
:0234F60033C1E0
:04375E006B8187CD27
:0234F80034C1DD
:043762006C8185CD24
:0234FA0035C1DA
:043766006D8183CD21
:0234FC0036C1D7
:04376A00A6DD81CD8A
:0234FE0037C1D4
:04376E00692D7FCD75
:0235000038C1D0
:0637720068816E7F92CD1C
:023502003AC1CC
:0637780069816E7F91CD16
:023504003CC1C8
:06377E006A816E7F90CD10
:023506003EC1C4
:063784006B816E7F8FCD0A
:0235080040C1C0
:06378A006C816E7F8ECD04
:02350A0042C1BC
:063790006D816E7F8DCDFE
:02350C0044C1B8
:0837960090DD6E7F0C947410AD
:02350E0047C1B3
:06379E00692D6E7F88CD4D
:0235100049C1AF
:0637A40068816D7F79CD04
:023512004BC1AB
:0637AA0069816D7F78CDFE
:023514004DC1A7
:0637B0006A816D7F77CDF8
:023516004FC1A3
:0637B6006B816D7F76CDF2
:0235180051C19F
:0637BC006C816D7F75CDEC
:02351A0053C19B
:0637C2006D816D7F74CDE6
:02351C0055C197
:0837C80077DD6D7F0C94741095
:02351E0058C192
:0637D000692D6D7F6FCD35
:023520005AC18E
:0637D60068816B7F60CDED
:023522005CC18A
:0637DC0069816B7F5FCDE7
:023524005EC186
:0637E2006A816B7F5ECDE1
:0235260060C182
:0637E8006B816B7F5DCDDB
:0235280062C17E
:0637EE006C816B7F5CCDD5
:02352A0064C17A
:0637F4006D816B7F5BCDCF
:02352C0066C176
:0837FA005EDD6B7F0C9474107E
:02352E0069C171
:06380200692D6B7F56CD1D
:023530006BC16D
:063808006881677F47CDD7
:023532006DC169
:06380E006981677F46CDD1
:023534006FC165
:063814006A81677F45CDCB
:0235360071C161
:06381A006B81677F44CDC5
:0235380073C15D
:063820006C81677F43CDBF
:02353A0075C159
:063826006D81677F42CDB9
:02353C0077C155
:08382C0045DD677F0C94741068
:02353E007AC150
:06383400692D677F3DCD08
:023540007CC14C
:06383A0068816F7E2ECDB7
:023542007EC148
:0638400069816F7E2DCDB1
:0235440080C144
:063846006A816F7E2CCDAB
:0235460082C140
:06384C006B816F7E2BCDA5
:0235480084C13C
:063852006C816F7E2ACD9F
:02354A0086C138
:063858006D816F7E29CD99
:02354C0088C134
:08385E002CDD6F7E0C94741048
:02354E008BC12F
:06386600692D6F7E24CDE8
:023550008DC12B
:06386C0068816F7D15CD9F
:023552008FC127
:0638720069816F7D14CD99
:0235540091C123
:063878006A816F7D13CD93
:0235560093C11F
:06387E006B816F7D12CD8D
:0235580095C11B
:063884006C816F7D11CD87
:02355A0097C117
:06388A006D816F7D10CD81
:02355C0099C113
:0838900013DD6F7D0C94741030
:02355E009CC10E
:06389800692D6F7D0BCDD0
:023560009EC10A
:06389E0068816F7BFCCC89
:02356200A0C106
:0638A40069816F7BFBCC83
:02356400A2C102
:0638AA006A816F7BFACC7D
:02356600A4C1FE
:0638B0006B816F7BF9CC77
:02356800A6C1FA
:0638B6006C816F7BF8CC71
:02356A00A8C1F6
:0638BC006D816F7BF7CC6B
:02356C00AAC1F2
:0838C200FADC6F7B0C9474101A
:02356E00ADC1ED
:0638CA00692D6F7BF2CCBA
:02357000AFC1E9
:0638D00068816F77E3CC74
:02357200B1C1E5
:0638D60069816F77E2CC6E
:02357400B3C1E1
:0638DC006A816F77E1CC68
:02357600B5C1DD
:0638E2006B816F77E0CC62
:02357800B7C1D9
:0638E8006C816F77DFCC5C
:02357A00B9C1D5
:0638EE006D816F77DECC56
:02357C00BBC1D1
:0838F400E1DC6F770C94741005
:02357E00BEC1CC
:0638FC00692D6F77D9CCA5
:02358000C0C1C8
:0639020068816160CACC7F
:02358200C2C1C4
:0639080069816160C9CC79
:02358400C4C1C0
:06390E006A816160C8CC73
:02358600C6C1BC
:063914006B816160C7CC6D
:02358800C8C1B8
:06391A006C816160C6CC67
:02358A00CAC1B4
:063920006D816160C5CC61
:02358C00CCC1B0
:08392600C8DC61600C94741010
:02358E00CFC1AB
:06392E00692D6160C0CCB0
:02359000D1C1A7
:0639340068816260B1CC65
:02359200D3C1A3
:06393A0069816260B0CC5F
:02359400D5C19F
:063940006A816260AFCC59
:02359600D7C19B
:063946006B816260AECC53
:02359800D9C197
:06394C006C816260ADCC4D
:02359A00DBC193
:063952006D816260ACCC47
:02359C00DDC18F
:08395800AFDC62600C947410F6
:02359E00E0C18A
:06396000692D6260A7CC96
:0235A000E2C186
:063966006881646098CC4A
:0235A200E4C182
:06396C006981646097CC44
:0235A400E6C17E
:063972006A81646096CC3E
:0235A600E8C17A
:063978006B81646095CC38
:0235A800EAC176
:06397E006C81646094CC32
:0235AA00ECC172
:063984006D81646093CC2C
:0235AC00EEC16E
:08398A0096DC64600C947410DB
:0235AE00F1C169
:06399200692D64608ECC7B
:0235B000F3C165
:06399800688168607FCC2D
:0235B200F5C161
:06399E00698168607ECC27
:0235B400F7C15D
:0639A4006A8168607DCC21
:0235B600F9C159
:0639AA006B8168607CCC1B
:0235B800FBC155
:0639B0006C8168607BCC15
:0235BA00FDC151
:0639B6006D8168607ACC0F
:0235BC00FFC14D
:0839BC007DDC68600C947410BE
:0235BE0002C247
:0639C400692D686075CC5E
:0235C00004C243
:0639CA006881606166CC1B
:0235C20006C23F
:0639D0006981606165CC15
:0235C40008C23B
:0639D6006A81606164CC0F
:0235C6000AC237
:0639DC006B81606163CC09
:0235C8000CC233
:0639E2006C81606162CC03
:0235CA000EC22F
:0639E8006D81606161CCFD
:0235CC0010C22B
:0839EE0064DC60610C947410AC
:0235CE0013C226
:0639F600692D60615CCC4C
:0235D00015C222
:0639FC00688160624DCC01
:0235D20017C21E
:063A0200698160624CCCFA
:0235D40019C21A
:063A08006A8160624BCCF4
:0235D6001BC216
:063A0E006B8160624ACCEE
:0235D8001DC212
:063A14006C81606249CCE8
:0235DA001FC20E
:063A1A006D81606248CCE2
:0235DC0021C20A
:083A20004BDC60620C94741091
:0235DE0024C205
:063A2800692D606243CC31
:0235E00026C201
:063A2E006881606434CCE5
:0235E20028C2FD
:063A34006981606433CCDF
:0235E4002AC2F9
:063A3A006A81606432CCD9
:0235E6002CC2F5
:063A40006B81606431CCD3
:0235E8002EC2F1
:063A46006C81606430CCCD
:0235EA0030C2ED
:063A4C006D8160642FCCC7
:0235EC0032C2E9
:083A520032DC60640C94741076
:0235EE0035C2E4
:063A5A00692D60642ACC16
:0235F00037C2E0
:063A6000688160681BCCC8
:0235F20039C2DC
:063A6600698160681ACCC2
:0235F4003BC2D8
:063A6C006A81606819CCBC
:0235F6003DC2D4
:063A72006B81606818CCB6
:0235F8003FC2D0
:063A78006C81606817CCB0
:0235FA0041C2CC
:063A7E006D81606816CCAA
:0235FC0043C2C8
:083A840019DC60680C94741059
:0235FE0046C2C3
:063A8C00692D606811CCF9
:023C000048CFAB
:043A9200A0DA03CCE7
:023C020049CFA8
:043A96009EDA03CCE5
:023C04004ACFA5
:043A9A009CDA03CCE3
:023C06004BCFA2
:043A9E009ADA03CCE1
:023C08004CCF9F
:043AA20098DA03CCDF
:023C0A004DCF9C
:043AA60096DA03CCDD
:043C0C00E3C94DCFEC
:043AAA0094DA03CCDB
:023C10004ECF95
:043AAE009BDAF5CBDF
:023C12004FCF92
:043AB20099DAF5CBDD
:023C140050CF8F
:043AB60097DAF5CBDB
:023C160051CF8C
:043ABA0095DAF5CBD9
:023C180052CF89
:043ABE0093DAF5CBD7
:023C1A0053CF86
:043AC20091DAF5CBD5
:043C1C00E4C953CFD5
:043AC6008FDAF5CBD3
:023C200054CF7F
:043ACA009ADBE7CBD1
:023C220055CF7C
:043ACE0098DBE7CBCF
:023C240056CF79
:043AD20096DBE7CBCD
:023C260057CF76
:043AD60094DBE7CBCB
:023C280058CF73
:043ADA0092DBE7CBC9
:023C2A0059CF70
:043ADE0090DBE7CBC7
:043C2C00E9CA59CFB9
:043AE2008EDBE7CBC5
:023C30005ACF69
:043AE60097DBD9CBC6
:023C32005BCF66
:043AEA0095DBD9CBC4
:023C34005CCF63
:043AEE0093DBD9CBC2
:023C36005DCF60
:043AF20091DBD9CBC0
:023C38005ECF5D
:043AF6008FDBD9CBBE
:023C3A005FCF5A
:043AFA008DDBD9CBBC
:043C3C00ECCA5FCFA0
:043AFE008BDBD9CBBA
:023C400060CF53
:043B020093DBCBCBBB
:023C420061CF50
:043B060091DBCBCBB9
:023C440062CF4D
:043B0A008FDBCBCBB7
:023C460063CF4A
:043B0E008DDBCBCBB5
:023C480064CF47
:043B12008BDBCBCBB3
:023C4A0065CF44
:043B160089DBCBCBB1
:043C4C00EECA65CF88
:043B1A0087DBCBCBAF
:023C500066CF3D
:043B1E008DDBBDCBB3
:023C520067CF3A
:043B22008BDBBDCBB1
:023C540068CF37
:043B260089DBBDCBAF
:023C560069CF34
:043B2A0087DBBDCBAD
:023C58006ACF31
:043B2E0085DBBDCBAB
:023C5A006BCF2E
:043B320083DBBDCBA9
:043C5C00EECA6BCF72
:043B360081DBBDCBA7
:023C60006CCF27
:043B3A0089DBAFCBA9
:023C62006DCF24
:043B3E0087DBAFCBA7
:023C64006ECF21
:043B420085DBAFCBA5
:023C66006FCF1E
:043B460083DBAFCBA3
:023C680070CF1B
:043B4A0081DBAFCBA1
:023C6A0071CF18
:043B4E007FDBAFCB9F
:043C6C00F0CA71CF5A
:043B52007DDBAFCB9D
:023C700072CF11
:043B560084DBA1CBA0
:023C720073CF0E
:043B5A0082DBA1CB9E
:023C740074CF0B
:043B5E0080DBA1CB9C
:023C760075CF08
:043B62007EDBA1CB9A
:023C780076CF05
:043B66007CDBA1CB98
:023C7A0077CF02
:043B6A007ADBA1CB96
:043C7C00F1CA77CF43
:043B6E0078DBA1CB94
:103C800005CB04CB03CB02CB01CB00CBFFCAFECAD2
:103C9000FBCAFACAF9CAF8CAF7CAF6CAF5CAF4CA18
:103CA000F1CAF0CAEFCAEECAEDCAECCAEBCAEACA58
:103CB000E7CAE6CAE5CAE4CAE3CAE2CAE1CAE0CA98
:103CC000DDCADCCADBCADACAD9CAD8CAD7CAD6CAD8
:103CD000D3CAD2CAD1CAD0CACFCACECACDCACCCA18
:103CE000C9CAC8CAC7CAC6CAC5CAC4CAC3CAC2CA58
:103CF000BFCABECABDCABCCABBCABACAB9CAB8CA98
:023D000038CFBA
:043B72006E7F93CB04
:023D020039CFB7
:043B76006E7F93CB00
:023D04003ACFB4
:043B7A006E7F93CBFC
:023D06003BCFB1
:043B7E006E7F93CBF8
:023D08003CCFAE
:043B82006E7F93CBF4
:023D0A003DCFAB
:043B86006E7F93CBF0
:023D0C003ECFA8
:043B8A006E7F0895AD
:023D0E003FCFA5
:043B8E006E7F91CBEA
:023D100040CFA2
:043B92006D7F83CBF5
:023D120041CF9F
:043B96006D7F83CBF1
:023D140042CF9C
:043B9A006D7F83CBED
:023D160043CF99
:043B9E006D7F83CBE9
:023D180044CF96
:043BA2006D7F83CBE5
:023D1A0045CF93
:043BA6006D7F83CBE1
:023D1C0046CF90
:043BAA006D7F08958E
:023D1E0047CF8D
:043BAE006D7F81CBDB
:023D200048CF8A
:043BB2006B7F73CBE7
:023D220049CF87
:043BB6006B7F73CBE3
:023D24004ACF84
:043BBA006B7F73CBDF
:023D26004BCF81
:043BBE006B7F73CBDB
:023D28004CCF7E
:043BC2006B7F73CBD7
:023D2A004DCF7B
:043BC6006B7F73CBD3
:023D2C004ECF78
:043BCA006B7F089570
:023D2E004FCF75
:043BCE006B7F71CBCD
:023D300050CF72
:043BD200677F63CBDB
:023D320051CF6F
:043BD600677F63CBD7
:023D340052CF6C
:043BDA00677F63CBD3
:023D360053CF69
:043BDE00677F63CBCF
:023D380054CF66
:043BE200677F63CBCB
:023D3A0055CF63
:043BE600677F63CBC7
:023D3C0056CF60
:043BEA00677F089554
:023D3E0057CF5D
:043BEE00677F61CBC1
:023D400058CF5A
:043BF2006F7E53CBC4
:023D420059CF57
:043BF6006F7E53CBC0
:023D44005DC060
:043E00006F7E50CAB7
:023D46005EC05D
:043E04006F7E50CAB3
:023D48005FC05A
:043E08006F7E50CAAF
:023D4A0060C057
:043E0C006F7E50CAAB
:023D4C0061C054
:043E10006F7E089524
:023D4E0062C051
:043E14006F7E4ECAA5
:023D500063C04E
:043E18006F7D40CAB0
:023D520064C04B
:043E1C006F7D40CAAC
:023D540065C048
:043E20006F7D40CAA8
:023D560066C045
:043E24006F7D40CAA4
:023D580067C042
:043E28006F7D40CAA0
:023D5A0068C03F
:043E2C006F7D40CA9C
:023D5C0069C03C
:043E30006F7D089505
:023D5E006AC039
:043E34006F7D3ECA96
:023D60006BC036
:043E38006F7B30CAA2
:023D62006CC033
:043E3C006F7B30CA9E
:023D64006DC030
:043E40006F7B30CA9A
:023D66006EC02D
:043E44006F7B30CA96
:023D68006FC02A
:043E48006F7B30CA92
:023D6A0070C027
:043E4C006F7B30CA8E
:023D6C0071C024
:043E50006F7B0895E7
:023D6E0072C021
:043E54006F7B2ECA88
:023D700073C01E
:043E58006F7720CA96
:023D720074C01B
:043E5C006F7720CA92
:023D740075C018
:043E60006F7720CA8E
:023D760076C015
:043E64006F7720CA8A
:023D780077C012
:043E68006F7720CA86
:023D7A0078C00F
:043E6C006F7720CA82
:023D7C0079C00C
:043E70006F770895CB
:023D7E007AC009
:043E74006F771ECA7C
:023D80007BC006
:043E7800616010CAAB
:023D82007CC003
:043E7C00616010CAA7
:023D84007DC000
:043E8000616010CAA3
:023D86007EC0FD
:043E8400616010CA9F
:023D88007FC0FA
:043E8800616010CA9B
:023D8A0080C0F7
:043E8C00616010CA97
:023D8C0081C0F4
:043E900061600895D0
:023D8E0082C0F1
:043E940061600ECA91
:023D900083C0EE
:043E9800626000CA9A
:023D920084C0EB
:043E9C00626000CA96
:023D940085C0E8
:043EA000626000CA92
:023D960086C0E5
:043EA400626000CA8E
:023D980087C0E2
:043EA800626000CA8A
:023D9A0088C0DF
:043EAC00626000CA86
:023D9C0089C0DC
:043EB00062600895AF
:023D9E008AC0D9
:043EB4006260FEC981
:023DA0008BC0D6
:043EB8006460F0C989
:023DA2008CC0D3
:043EBC006460F0C985
:023DA4008DC0D0
:043EC0006460F0C981
:023DA6008EC0CD
:043EC4006460F0C97D
:023DA8008FC0CA
:043EC8006460F0C979
:023DAA0090C0C7
:043ECC006460F0C975
:023DAC0091C0C4
:043ED000646008958D
:023DAE0092C0C1
:043ED4006460EEC96F
:023DB00093C0BE
:043ED8006860E0C975
:023DB20094C0BB
:043EDC006860E0C971
:023DB40095C0B8
:043EE0006860E0C96D
:023DB60096C0B5
:043EE4006860E0C969
:023DB80097C0B2
:043EE8006860E0C965
:023DBA0098C0AF
:043EEC006860E0C961
:023DBC0099C0AC
:043EF0006860089569
:023DBE009AC0A9
:043EF4006860DEC95B
:023DC0009BC0A6
:043EF8006061D0C96C
:023DC2009CC0A3
:043EFC006061D0C968
:023DC4009DC0A0
:043F00006061D0C963
:023DC6009EC09D
:043F04006061D0C95F
:023DC8009FC09A
:043F08006061D0C95B
:023DCA00A0C097
:043F0C006061D0C957
:023DCC00A1C094
:043F1000606108954F
:023DCE00A2C091
:043F14006061CEC951
:023DD000A3C08E
:043F18006062C0C95A
:023DD200A4C08B
:043F1C006062C0C956
:023DD400A5C088
:043F20006062C0C952
:023DD600A6C085
:043F24006062C0C94E
:023DD800A7C082
:043F28006062C0C94A
:023DDA00A8C07F
:043F2C006062C0C946
:023DDC00A9C07C
:043F3000606208952E
:023DDE00AAC079
:043F34006062BEC940
:023DE000ABC076
:043F38006064B0C948
:023DE200ACC073
:043F3C006064B0C944
:023DE400ADC070
:043F40006064B0C940
:023DE600AEC06D
:043F44006064B0C93C
:023DE800AFC06A
:043F48006064B0C938
:023DEA00B0C067
:043F4C006064B0C934
:023DEC00B1C064
:043F5000606408950C
:023DEE00B2C061
:043F54006064AEC92E
:023DF000B3C05E
:043F58006068A0C934
:023DF200B4C05B
:043F5C006068A0C930
:023DF400B5C058
:043F60006068A0C92C
:023DF600B6C055
:043F64006068A0C928
:023DF800B7C052
:043F68006068A0C924
:023DFA00B8C04F
:043F6C006068A0C920
:023DFC00B9C04C
:043F700060680895E8
:023DFE00BAC049
:103F740060689EC960E00895162F0E94160F602F96
:103F840040FBF6E4E02F449140F90895062F19818F
:103F94000E94140F0895DB010981F894BBB928B875
:103FA400ABB938B80BB958B8789468B81196088189
:103FB400F894BBB928B8ABB938B80BB958B87894E9
:103FC40068B80895DB010B81F894BBB928B8ABB984
:103FD40038B80BB958B8789468B811960A81F8942F
:103FE400BBB928B8ABB938B80BB958B8789468B825
:103FF4000895DB01F894BBB928B8ABB938B8EBB86D
:1040040058B8789468B81196F894BBB928B8ABB985
:1040140038B8FBB858B8789468B808950D811C81F5
:10402400889440FD0894601F0FB7711F1FB76D83FC
:104034007C83012340E010FB40F913FB42F915FB9C
:1040440044F901FB46F912FB47F908950D811C81DF
:104054000617889440FD0894060B170B0D831C83E8
:104064000FB742E000FB40F903FB42F905FB44F9BA
:1040740001FB46F902FB47F9089500E00919902E67
:104084000FB7F6E4E92D449100FB40F905FB44F930
:1040940003FB42F9426008950C8903FB02F90C8B7F
:1040A4000C94A0100C890C7F0C8B08950C890C7F48
:1040B40001600C8B08950C890C7F02600C8B0895B1
:1040C4009A8801C09B8840FBF6E4E92D449140F9AD
:1040D4000C8903FB42F908959A8A08959B8A0895EE
:1040E4006295762F607F7F70092D0F70602B092DEC
:1040F400007F072B902E40FBF6E4E92D449140F914
:104104000895762F607F7F70092D0F70602B629564
:10411400092D007F072B902E40FBF6E4E92D4491F6
:1041240040F90895BC81AD810E944907FD01BA811F
:10413400AB810E94570778816981497E6150704044
:1041440009F04460698378830895ECDF3196119611
:10415400AB83BA83ED83FC830895E4DF3197119731
:10416400AB83BA83ED83FC830895EFDF42FDFDCF7B
:104174000895F3DF42FF089502970895BC81AD814D
:10418400F881E9814B7242600E94490790160AF453
:10419400406809F440640DF44061319709F04460CB
:1041A400E983F8830895EADF1196AD83BC8308950B
:1041B400E5DF1197AD83BC830895F5DF46FD0895CF
:1041C40042FF089502970895F3DF46FD089542FFE4
:1041D4000895029708954F7B426019810E94160F3B
:1041E400BC81AD810E94570708810A95088309F4B0
:1041F40040640895F0DF1196AD83BC830895EBDF2E
:104204001197AD83BC830895F5DF46FD08950297A9
:104214000895F5DF46FD0895029708954F7B4260A7
:104224000E94490719810E94140F08810A95088386
:1042340009F440640895BC81AD811196AD83BC83BB
:104244001197ECDF0895BC81AD811197AD83BC83D8
:104254001196E4DF0895EFDF46FD0895029708956F
:0A426400F2DF46FD08950297089569
:1044000008950895089508950895089508950895C4
:1044100008950895089508950895089508950895B4
:1044200008950895089508950895089508950895A4
:104430000895089508950895089508950895089594
:104440000895089508950895089508950895089584
:104450000895089508950895089508950895089574
:104460000895089508950895089508950895089564
:104470000895089508950895089508950895089554
:02448000F6CE76
:06426E00698185DE14C821
:02448200F8CE72
:0442740068818CCE03
:02448400F9CE6F
:064278000E94C00FE9CE18
:02448600FBCE6B
:06427E000E9425108BCE0A
:0A448800FACD08CE0DCE26CEF9CEF7
:0642840069817ADE0BC81F
:02449200FBCE5F
:04428A00698181CEF7
:02449400FCCE5C
:06428E000E94C00FC6CE25
:02449600FECE58
:0C4294000E9425100E94D9110C945310B8
:0A449800F2CD00CE05CE20CEFFCEFF
:0842A00069816CDE0C945219D7
:0244A20002CF47
:0442A8006A8172CEE7
:0244A40003CF44
:0642AC000E94C30FCFCEFB
:0244A60005CF40
:0642B2000E94251088CED9
:0A44A800EACDF8CD01CE0ACE03CF15
:0842B800698160DE0C945419C9
:0244B20006CF33
:0442C0006B8166CEDA
:0244B40007CF30
:0642C4000E94C30FABCE07
:0244B60009CF2C
:0C42CA000E9425100E94D9110C9456107F
:0A44B800E2CDF0CDFECD04CE0ACF18
:0842D600698151DE0C945619B8
:0244C2000DCF1C
:0442DE006C8157CECA
:0244C4000ECF19
:0642E2000E94C60FB4CEDD
:0244C60010CF15
:0442E8000C949D1382
:0844C800DACDE8CDEDCD0ECFF9
:0A42EC000E945C190ADF0C947410A4
:0244D00012CF09
:0842F600698141DE0C945819A6
:0244D20015CF04
:0442FE006D8147CEB9
:0244D40016CF01
:064302000E94C60F8CCEE4
:0244D60018CFFD
:044308000C94B2134C
:0844D800D2CDE0CDE5CD16CFF9
:0A430C000E945C19E9DE0C947410A5
:0244E0001ACFF1
:04431600698131CEBA
:0244E2001BCFEE
:04431A002EDE39CE8C
:0244E4001CCFEB
:04431E00B70197CE7E
:0244E6001DCFE8
:064322000E94251067CE89
:0A44E800CACDD8CDE1CD08951BCF59
:08432800698128DE0C945A198A
:0244F2001ECFDB
:04433000692D2ECEF7
:0244F4001FCFD8
:04433400B70174CE8B
:0244F60020CFD5
:0C4338000E9425100E94D9110C949510D1
:1044F800C2CDD0CDDECD08950895089508950895CC
:1045080008950895089508950895089508950895BB
:1045180008950895089508950895089508950895AB
:10452800089508950895089508950895089508959B
:10453800089508950895089506CE33CE59CE79CEBC
:10454800089508950895089506CE30CE56CE79CEB2
:10455800089508950895089506CE2DCE53CE79CEA8
:10456800089508950895089502CE2CCE50CE76CEA3
:10457800089508950895089508950895089508954B
:10458800089508950895089508950895089508953B
:10459800089508950895089508950895089508952B
:1045A800089508950895089508950895089508951B
:1045B800089508950895089508950895089508950B
:1045C80008950895089508950895089508950895FB
:1045D80008950895089508950895089508950895EB
:1045E80008950895089508950895089508950895DB
:1045F80008950895089508954400000400040400EF
:10460800080C0C080C08080C000404000400000442
:104618000C08080C080C0C08202424202420202432
:104628002C28282C282C2C28242020242024242022
:10463800282C2C282C28282C000404000400000412
:104648000C08080C080C0C08040000040004040002
:10465800080C0C080C08080C2420202420242420F2
:10466800282C2C282C28282C2024242024202024E2
:104678002C28282C282C2C288084848084808084D2
:104688008C88888C888C8C888480808480848480C2
:10469800888C8C888C88888CA4A0A0A4A0A4A4A0B2
:1046A800A8ACACA8ACA8A8ACA0A4A4A0A4A0A0A4A2
:1046B800ACA8A8ACA8ACACA8848080848084848092
:1046C800888C8C888C88888C808484808480808482
:1046D8008C88888C888C8C88A0A4A4A0A4A0A0A472
:1046E800ACA8A8ACA8ACACA8A4A0A0A4A0A4A4A062
:0846F800A8ACACA8ACA8A8AC6A
:00000001FF
